:0200000480007A
:100000006F000005732F2034930F80006308FF03F7
:10001000930F90006304FF03930FB0006300FF038E
:10002000130F000063040F0067000F00732F2034CC
:1000300063540F006F00400093E19153171F0000BD
:1000400023223FFC171F000023200FFC6FF01FFF2F
:100050009300000013010000930100001302000050
:100060009302000013030000930300001304000038
:100070009304000013050000930500001306000020
:100080009306000013070000930700001308000008
:10009000930800001309000093090000130A0000F0
:1000A000930A0000130B0000930B0000130C0000D8
:1000B000930C0000130D0000930D0000130E0000C0
:1000C000930E0000130F0000930F0000732540F102
:1000D0006310050097020000938202017390523072
:1000E000735044749702000093820201739052305F
:1000F00073500018970200009382020273905230EE
:10010000B70200809382F2FF7390023B9302F001EA
:100110007390023A7350403097020000938242017C
:100120007390523073502030735030309301000080
:1001300097020000938242ED739052301305100035
:100140001315F501634C05000F00F00F930110002B
:100150009308D0051305000073000000970200000B
:100160009382821E638A020073905210B7B200001D
:100170009382921073902230735000303715000034
:1001800013050580732005301305200273203530D8
:10019000970200009382420173901234732540F15C
:1001A0007300203093014001731000147325001474
:1001B00093030000631075169301500173550014EA
:1001C00073D507149303000063167514930160013F
:1001D00073600814732500149303F001631C7512F7
:1001E00073D0011493012000732500149303300091
:1001F0006312751293013000F3F50014930330007D
:10020000639A7510930140007366021493032000F3
:100210006312761093015000F356011493036000AB
:10022000639A760E930160003725AD0B1305A5DEAA
:10023000F315051493032000639E750C9301700061
:10024000372500001305A5DEF3350514B723AD0BE4
:100250009383A3DE6390750C9301800037C5000083
:100260001305F5EEF3250514B703AD0B6394750A7A
:10027000930190003725AD0B1305A5DE731505140A
:10028000B7C3AD0B9383F3EE631675089301A0001B
:10029000372500001305A5DE73350514B723AD0B14
:1002A0009383A3DE631875069301B00037C5000081
:1002B0001305F5EE73250514B703AD0B631C750428
:1002C0009301C00073250014B7C3AD0B9383F3EE05
:1002D000631275049302001073B0021097020000BD
:1002E0009382020173901214730020109301F000A6
:1002F0001300000093030000631E70000F00F00F56
:10030000930110009308D00513050000730000004E
:10031000631030020F00F00F638001009391110011
:1003200093E111009308D0051385010073000000CC
:100330000F00F00F930110009308D0051305000083
:10034000730000009302D00063E651009302F000B6
:1003500063F23202F322201413038000E39C62FA5A
:100360000F00F00F930110009308D0051305000053
:1003700073000000F322201413032000E39C62F8B2
:10038000F322101493824200739012147300201011
:10039000731000C00000000000000000000000001A
:1003A000000000000000000000000000000000004D
:1003B000000000000000000000000000000000003D
:1010000000000000000000000000000000000000E0
:1010100000000000000000000000000000000000D0
:1010200000000000000000000000000000000000C0
:1010300000000000000000000000000000000000B0
:081040000000000000000000A8
:1020000001000000000000000000000000000000CF
:040000058000000077
:00000001FF
